:02000000452891
:020008001028BE
:04000A00003400348A
:10002000F40003088301F5000A08F6008A010B1C9E
:100030001B28AC240B100B1D3F280B11EE30831234
:1000400003138100861D26280430860683160313B9
:10005000EC0B3F2883160313E30B2F287715F719B2
:100060003B288D2083120313A4002626C020831270
:100070000313A7002E26C83083160313EC0076085E
:100080008A00750883007408090030308312031356
:10009000A4002626803083120313A7002E26F70122
:1000A000F801C624C83083160313EC00831603132B
:1000B0003F308500F030860006309F008312031326
:1000C000F2308600810183160313640081128111CE
:1000D000011581100110811383120313EE3081008A
:1000E0008B168B150B128B178D2083120313A40014
:1000F0002626C02083120313A7002E26F81B3623C2
:10010000781B8D25F81AC725AC24781ADD25AC2478
:0A01100078187E28630000007E28A6
:06011A008312031386109E
:1001200041309F008316031304309F008312031392
:1001300000000000000000000000000000000000BF
:1001400000000000000000000000000000000000AF
:1001500000000000000000001F151F19AD288614C4
:1001600040309F008316031306309F008312031351
:100170001E0883160313ED0003106D0C143E0800D7
:1001800083120313861049309F0083160313043033
:100190009F00831203130000000000000000000015
:1001A000000000000000000000000000000000004F
:1001B00000000000000000000000000000001F150B
:1001C0001F19E028861440309F0083160313063061
:1001D0009F00831203131E0883160313ED00031000
:0601E0006D0C403E08001A
:10020000E03E3F3983160313EA0001308A006A0892
:1002100082070034003400340034003400340034E9
:1002200000340034003468342A34733400346A34BF
:1002300029343F343E343C34383430342034213493
:10024000233427342F340034003400343134003464
:100250004C34003406341134153409340234143467
:100260000B34103404341E340D3412340734053486
:100270000F3416341B340A34083403340C34183465
:100280000E3419341D341334003400340034003477
:10029000003483160313EA0001308A006A08801BC9
:1002A0003F3482073F343F34453454344934413479
:1002B0004E344D34533455345234573444344B3423
:1002C00047344F344834563446343F344C343F344A
:1002D00050344A3442345834433459345A34513403
:1002E0003F343F34353434343F3433343F343F3497
:1002F0003F3432343F343F342B343F343F343F3487
:100300003F34313436343D342F343F343F343F347E
:100310003F343F3437343F343F343F3438343F3454
:10032000393430343F343F343F343F343F342A345F
:100330003F343F343F343F343F343F343F343F3425
:100340003F343F343F343F343F343F343F342E3426
:100350003F343F343F343F343F343F343F343F3405
:100360003F343F343F343F343F343F343F343F34F5
:100370003F343F343F343F343F343F343F343F34E5
:100380003F343F343F343F343F342C343F343F34E8
:100390003F343F343F343F343F343F343F343F34C5
:0403A0003F343F3473
:10040000EC3E83160313EB0002308A006B08820770
:10041000FB34EF34E434DA34D134C834C134BA3480
:10042000B334AD34A734A2349C34983493348F342D
:100430008B348734843480347D347A347734743424
:1004400072346F346D346A346834663464346234C0
:1004500060345E345D345B3459345834563455342A
:100460005334523451344F344E344D344C344A3476
:1004700049344834473446344534443443344234B0
:100480004234413440343F343E343E343D343C34D5
:100490003B343B343A3439343934383437343734F4
:1004A000363436343534343434343334333432340B
:1004B000323431343134303430342F342F342E341C
:1004C0002E342E342D342D342C342C342C342B3427
:1004D0002B342A342A342A34293429342934283430
:1004E0002834283427342734273426342634263435
:1004F0002634253425342534243424342434243437
:100500002334233423342334223422342234223437
:1005100083160313EA00EA1F902A6A1FB32A002BEE
:1005200083160313EA0002308A006A083F39820703
:10053000433451342034433451342034433451341F
:1005400020344434453420344D3430344B34473433
:100550004B3420344D3430344B3447344B34203416
:100560002B344B34003483160313EA0002308A0024
:100570006A083F39820743345134203443345134BC
:1005800020344334513420344434583420344334F8
:1005900051342034433451342034433451342034E2
:1005A0004434583420344434453420344D343034C9
:1005B0004B3447344B3420344D3430344B3447348F
:0A05C0004B3420342B344B3400344C
:1006000083160313EA0003308A006A083F39820721
:10061000433451342034433451342034433451343E
:100620002034543445345334543420344334513416
:10063000203443345134203443345134203454343E
:1006400045345334543420344434453420344D3408
:1006500030344B3447344B3420344D3430344B3405
:0C06600047344B3420342B344B3400342E
:04066C00F813F71177
:1006700077144B30A6255924F81B652B83160313DA
:10068000E100003C0319542C831603136108023C5B
:100690000319652B6108043C0319662B6108073CAC
:1006A0000319702B61080A3C0319AB2B6108083C45
:1006B0000319F12B6108033C0319322C6108193C22
:1006C0000319432C3F30A625362B542C4D30A6253C
:1006D000831203132A08303EA6252030A625362B88
:1006E0004E30A625592483160313E100003C03195C
:1006F000542C61082F3C0319A02B6108023C0319FC
:10070000A02B6108033C0319A02B6108273C0319A7
:10071000A22B6108043C0319A22B6108073C0319B2
:10072000A22B6108233C0319A42B6108083C031980
:10073000A42B61080F3C0319A42B3F30A625702B76
:100740000130A52B0230A52B033083120313AA001E
:100750003A25C624362B5230A625F715A030840042
:10076000403083160313E700831603138001840AC5
:1007700083160313E70BB42B403083160313E700F3
:10078000A030840083160313E801592400380319AC
:10079000EF2B0038031DD12B83160313E80A2030FA
:1007A000D62B83160313E801E900492183160313AE
:1007B0008000840A83160313E70BDF2BEC2B6808F9
:1007C000023C031CE52B7324C92B8403840383168A
:1007D0000313800183120313F7115325362BF711EE
:1007E000542C83160313E401E50183120313240838
:1007F00083160313E6002830E602031C012CE40AEA
:10080000FC2BE6070430E602031C082CE50A032C47
:10081000E6076408003C0319102C6408303EA62546
:10082000831603136508303EA62583160313660856
:10083000003C03192F2C2E30A62583160313E60B3C
:10084000262C3230A6253530A6252F2CE60B2B2C56
:100850003530A6252F2C3730A6253530A62520305B
:10086000A625362B831203132B183C2C2B1459303E
:10087000A6252030A625412C2B104E30A625203051
:10088000A6253A25362B831203132B194D2C2B1535
:100890004C30A6252030A625522C2B115230A625EF
:1008A0002030A6253A25362B4530A625F8017710AD
:1008B00008002B3083160313E3007711732483168B
:1008C0000313E1000038031D6A2CF81B6A2C77190A
:1008D0006E2C5E2C8316031361080800003083160B
:1008E0000313E1000800013083160313E000E20166
:1008F000F81BAA2CAC24F81E852CC72503148316DC
:100900000313E00D2B30E300E201AC24781E902CA1
:10091000DD25031083160313E00D2B30E300E20105
:10092000AC247818782CF12583160313E20A6008AA
:10093000013C031DA02C6208043C031CAA2C782C4B
:10094000831603136208003C0318782C83160313E4
:100950006008080000300800831203132B1DBB2C15
:10096000831203130608F03AC039F800061EF81681
:10097000861E7816C12C831203130608F03AF0394C
:0C098000F800781A7814F81A78140800AF
:04098C000830F3003C
:100990008312031328308400F00170082525831288
:1009A00003138000F00A840AF30BCD2C8312031387
:1009B0002A080319032D033C031C032D25302A06A6
:1009C0002B062802031D032D64302A072B0729025A
:1009D000031D032D831203132A08F0000310F00DEA
:1009E000F00DF00DF00DF00DF00D4030F300A030E3
:1009F000840070082525831603138000840AF00AFA
:100A0000F30BF92C0800013083120313AA00013004
:100A1000AB0083160313A00138250430F300F30B59
:100A2000122D242D7308F000F00E0310F00DF00DC0
:100A30007008882200380319212DF1006E25F00A74
:100A4000182DF1016E250F2DEA2CF0000308F2009D
:100A50007008831203178D00831603178C130C1470
:100A6000831203170C08F100720883007108080054
:100A70003A25532D8312031325302A062B06A8008E
:100A800064302A072B07A900283084000830F300BF
:100A9000F001831203130008F1006E25840AF00AA6
:100AA000F30B492D0800831203132A08F0000310EA
:100AB000F00DF00DF00DF00DF00DF00D4030F300E5
:100AC00083160313A0308400831603130008F1007B
:100AD0006E25840AF00AF30B642D08000308F20067
:100AE000831603178C18722D8312031770088D005C
:100AF00071088C00831603178C130C158B1355305B
:100B00008D00AA308D008C148B170C1183160317DF
:0A0B10008C18882D7208830008007D
:060B1A00F7147813A0306F
:100B20008400831203134030A3007808031DA32D13
:100B30008316031300080319A32DA625840A831224
:100B40000313A30B952DF801F71008000021831261
:100B50000313A1002108003C031DB42DF125F1254C
:100B6000F125F125F1250800831203132108013C2A
:100B70000319C42D211CBE2DC725BF2DDD25031053
:100B800083120313A10CB42DF125F1250800771869
:100B9000CC2D8312031306147718D22D831203135E
:100BA0002B1CD52D831203138615F125F125002664
:100BB0008312031386110610152E7718E22D831267
:100BC000031306147718E82D831203132B1CEB2D47
:100BD0008312031386150026831203138611061051
:100BE000152E831203132008A5008030A6000000F4
:100BF000000000000000A60BF72DA50BF52D080046
:100C000083120313200883120313A5008312031316
:100C1000270883120313A600000000000000000054
:100C2000A60B0C2EA50B062E08008312031320081A
:100C300083120313A5002208A60000000000000094
:100C40000000A60B1D2EA50B1B2E080083120313FC
:100C50002408002283120313A00008008312031348
:0C0C60002708003C83120313A2000800C8
:02400E00313D42
:00000001FF
